:10000000B4C0CEC0CDC0CCC0CBC0CAC0C9C0C8C0AF
:10001000C7C0C6C0C5C0C4C0C3C0C2C0C1C0C0C0C4
:10002000BFC0BEC0BDC053756D3A0048656C643A30
:100030000057494E4E45522100736563004E6F20B4
:100040004D617463682100596F75206172650A0003
:10005000506C656173650A7363616E20746167003B
:100060004C657420676F0A3D207265706C61790081
:10007000546167204944203E0A003C2053636F725C
:1000800065730A0047414D454F5645520A4E6F2051
:1000900057696E2E00203E00202047616D650A20C2
:1000A000204F76657200310A7365632E2E2E003262
:1000B0000A736563732E2E2E00330A736563732EE5
:1000C0002E2E00526573746F72650A677269702014
:1000D0006E6F77004E6F20526F6F6D0A666F7220E1
:1000E000796F7521005363616E207461670A005453
:1000F000696D654C656674004D495353494F4E0A0E
:1001000020535441525421005363616E0A41444DBF
:10011000494E2E2E2E004E6F206D6F72650A526F63
:100120006F6D21203A280057656C636F6D650A007A
:100130000A65786973747321005363616E20610AE4
:10014000746167206E6F770047616D6520476F3E71
:10015000003C416464205461670A00204A616220C7
:10016000616E0A2045796521000011241FBECFE58C
:10017000D4E0DEBFCDBF10E0A0E6B0E0EAE7F1E1F9
:1001800002C005900D92A23CB107D9F711E0A2EC94
:10019000B0E001C01D92AB3CB107E1F71ED1ECC746
:1001A0002FCF8E9A969A8CE792E90197F1F796985D
:1001B00084ED90E30197F1F708958E9A969A8EE375
:1001C00099E40197F1F796988AE698E10197F1F79B
:1001D00008958E9A969A20E137E289E190E001979E
:1001E000F1F721503040C9F7969884ED90E30197DC
:1001F000F1F70895CF93DF938E9A969A8EE399E460
:10020000FC013197F1F79698ECE4FDE1DF011197DD
:10021000F1F7969ADC011197F1F79698DF011197A3
:10022000F1F7969ADC011197F1F79698A8EAB1E6F2
:10023000ED012197F1F7969AEC012197F1F7969845
:10024000EF012197F1F7969AEC012197F1F7969833
:10025000EF012197F1F7969AEC012197F1F7969823
:10026000ED012197F1F7969AEC012197F1F7969815
:10027000EF012197F1F7969AEC012197F1F7969803
:100280003197F1F7969A0197F1F796981197F1F750
:10029000DF91CF9108955D9BFECF8CB908955F9B50
:1002A000FECF8CB190E00895FC0104C05D9BFECFB1
:1002B0008CB9319680818823C9F70895FC0104C068
:1002C0005D9BFECF31968CB984918823C9F7089540
:1002D000B89AC0980895B89AC09A08955D9BFECFC9
:1002E0008EEF8CB95D9BFECF88E58CB90895982F71
:1002F0005D9BFECF8EEF8CB95D9BFECF87E48CB902
:100300005D9BFECF9CB95D9BFECF6CB90895B89AFA
:10031000C098892B21F45F9BFECF8CB105C05F9BF9
:10032000FECF8CB18A30D9F78093BE015F9BFECFA0
:100330008CB18093BF015F9BFECF8CB18093C001D5
:100340005F9BFECF8CB18093C1015F9BFECF8CB1D0
:100350008093C2015F9BFECF8CB18093C3015F9BF2
:10036000FECF8CB18093C4015F9BFECF8CB1809394
:10037000C5015F9BFECF8CB18093C6015F9BFECF12
:100380008CB18093C7015F9BFECF8CB18093C80175
:100390005F9BFECF9CB19093C901B89AC09A80919F
:1003A000BE018A3019F060E670E004C09D3041F073
:1003B00069E670E08EEB91E074D681E090E00895FC
:1003C000EEEBF1E08181819381E0E83CF807D1F721
:1003D0001092C80180E090E008952F923F924F92D2
:1003E0005F926F927F928F929F92AF92BF92CF92C5
:1003F000DF92EF92FF920F931F93CF93DF93CDB7CE
:10040000DEB72B970FB6F894DEBF0FBECDBF8AB113
:1004100088618AB986E080BD89E189B910BC20E194
:1004200037E289E190E00197F1F721503040C9F7B8
:100430005D9BFECF8EEF8CB95D9BFECF84E48CB9C3
:100440005D9BFECF8EEF8CB95D9BFECF82E58CB9B4
:100450005D9BFECF8EEF8CB95D9BFECF8BE48CB99C
:100460005D9BFECF8EEF8CB95D9BFECF84E58CB992
:100470005D9BFECF8EEF8CB95D9BFECF89E98CB979
:100480005D9BFECF88E38CB95D9BFECF8EEF8CB970
:100490005D9BFECF80E58CB95D9BFECF8FE78CB96D
:1004A0001DDF5D9BFECF8EEF8CB95D9BFECF88E696
:1004B0008CB9B998BA988BE591E000DF36B3327009
:1004C00026B3247084EC99E00197F1F7332339F0D7
:1004D0002223A1F71092C2003093C30004C02093DE
:1004E000C2001092C30036B3327026B3247084EC7D
:1004F00099E00197F1F73323B1F32223A1F320937D
:10050000C2003093C300ECE48E2EE1E09E2E7EEB21
:10051000A72E71E0B72E65E3262E61E0362E57E256
:10052000452E51E0552E46E1642E41E0742ED6DE74
:1005300081E591E0C3DE88E491E0C0DE36B332703D
:1005400026B3247084EC99E00197F1F7332321F06E
:10055000222309F4B1C0F2CF2093C2001092C3004D
:10056000BDDE89E391E0AADE34DE80E090E006C0E3
:1005700084E294EF0197F1F781E090E0C8DE892BE7
:10058000B9F70FDE0EDE0DDE8401EE24FF24B50187
:10059000C8017ED5009721F4F092BD01E092BC0124
:1005A0000894E11CF11C2AE0E216F10429F0055F31
:1005B0001F4F892B19F0EBCF892B09F58FDEE091C6
:1005C000BC01F091BD01EE0FFF1FEB5CFE4F80817F
:1005D000918123E0880F991F2A95E1F78F589F4F4B
:1005E00063DE80E391E06ADE28EA31E689E190E0AB
:1005F0000197F1F72150304009F466C0F7CF84012C
:100600007101CC24DD24F8018081882319F080E079
:1006100090E033C0B501C80144D5D092BD01C0926D
:10062000BC0180914A0190914B01F7019183808335
:10063000019690934B0180934A0150DEC2013EDE49
:10064000E091BC01F091BD01EE0FFF1FEB5CFE4F8E
:1006500080819181B3E0880F991FBA95E1F78F5897
:100660009F4F22DE28EA31E689E190E00197F1F719
:1006700021503040C9F781E090E00894C11CD11CA2
:10068000FAE0CF16D10449F0055F1F4F22E030E0B9
:10069000E20EF31E892BC1F4B6CF892BA9F41EDE1E
:1006A000C3010CDE28EA31E689E190E00197F1F719
:1006B0002150304049F0F8CF1092C2003093C3006F
:1006C0008CE792E90197F1F78091C200882309F045
:1006D0002ECFAEEB8A2EA1E09A2EF2E04F2EF1E063
:1006E0005F2EECE46E2EE1E07E2E71E2272E71E0AB
:1006F000372E109249011092BB011092BA0110924C
:10070000D9001092D80080E090E0FC01EC53FF4F3C
:1007100011821082FC01E35FFE4F11821082FC0106
:10072000EF5DFE4F11821082FC01E251FF4F1182FA
:100730001082FC01E652FF4F118210820296843132
:10074000910519F7CBDD88E091E0B8DD42DD80E06E
:1007500090E006C084E294EF0197F1F781E090E029
:10076000D6DD5C01892BB1F71CDD1BDD1ADDB40180
:10077000C20197D4B3DD88EF90E0A0DD28EA31E62E
:1007800089E190E00197F1F72150304009F4E4C18C
:10079000F7CFA4DD8FEE90E091DD86B38270809379
:1007A000C30086B384708093C200E0E0F0E04AC0EA
:1007B00020E43FE189E190E00197F1F721503040DA
:1007C000C9F73196E530F10521F4EBDCE0E0F0E02B
:1007D00004C080E593EC0197F1F72091D8003091A7
:1007E000D9002F5F3F4F3093D9002093D8005D9BF5
:1007F000FECF8EEF8CB95D9BFECF8CE78CB95D9BF5
:10080000FECF81E08CB95D9BFECF82E08CB95D9B11
:10081000FECF1CB8C90166E170E087D45D9BFECFB6
:1008200088E2861B8CB92558334024F081E0809300
:10083000490112C086B382708093C30086B384706E
:100840008093C2008091C300882309F0B1CF8091CA
:10085000C200882309F0ACCF80914901813009F4AE
:1008600080C13CDD85EE90E029DDB3DC80E090E0E6
:1008700006C084E294EF0197F1F781E090E047DD54
:10088000892BB9F78EDC8DDC8CDC4AE050E0B401BA
:10089000C2010ED4892B21F481E08093490161C10A
:1008A0008301EE24FF24B401C801F2D3009721F4A0
:1008B000F092BD01E092BC010894E11CF11CEAE059
:1008C000EE16F10429F0055F1F4F892BD9F1EBCF0C
:1008D000892BC1F1830165E3E62E61E0F62ECC247D
:1008E000DD24F8018081882319F080E090E015C0B4
:1008F000B401C801D6D3D092BD01C092BC01809191
:100900004A0190914B01F701918380830196909366
:100910004B0180934A0181E090E00894C11CD11CF6
:10092000FAE0CF16D10449F0055F1F4F22E030E016
:10093000E20EF31E892B31F4D4CF892B19F484ED08
:1009400090E08AC3CBDCE091BC01F091BD01EE0FD9
:10095000FF1FEB5CFE4F8081918143E0880F991F60
:100960004A95E1F78F589F4F9FDC86B38270809342
:10097000C30096B394709093C200882319F499230E
:1009800009F450C020E137E289E190E00197F1F7E6
:1009900021503040C9F7A2DC83EC90E08FDC20E1ED
:1009A00037E289E190E00197F1F721503040C9F733
:1009B00095DC89EB90E082DC20E137E289E190E090
:1009C0000197F1F721503040C9F788DC8FEA90E0B9
:1009D00075DC20E137E289E190E00197F1F72150E1
:1009E0003040C9F77BDC86EA90E068DC20E137E242
:1009F00089E190E00197F1F721503040C9F76EDCB2
:100A0000E091BC01F091BD01EE0FFF1FEB5CFE4FCA
:100A10008081918123E0880F991F2A95E1F78F58F3
:100A20009F4F42DCE091BC01F091BD01EE0FFF1F32
:100A3000DF01A652BF4F8D919C91119701968D9326
:100A40009C93EC53FF4F1182108270C08091D800AC
:100A50009091D90001969093D9008093D80020916D
:100A6000BC013091BD01220F331FF901EC53FF4F40
:100A7000408151814F5F5F4F51834083F901E35FB4
:100A8000FE4F80819181019691838083F901EF5D12
:100A9000FE4F808191818417950714F45183408320
:100AA0008091BA019091BB01841795077CF4509313
:100AB000BB014093BA0181DB28E233E289E190E097
:100AC0000197F1F72150304051F0F8CF20E137E2A3
:100AD00089E190E00197F1F721503040C9F75D9B23
:100AE000FECF8EEF8CB95D9BFECF8CE78CB95D9B02
:100AF000FECF81E08CB95D9BFECF82E08CB95D9B1F
:100B0000FECF1CB82091D8003091D900C90166E110
:100B100070E00BD35D9BFECF88E2861B8CB9255815
:100B2000334024F081E08093490111C086B3827084
:100B30008093C30086B384708093C2008091C30009
:100B4000882329F48091C200882309F47FCF41DBF8
:100B500080914901813029F080914901882309F46D
:100B600018CEF30100E010E08081882311F00F5FC0
:100B70001F4F3B9691E0EA3BF907B1F7AEEEB0E0CC
:100B8000A10126C011961C930E93710160E070E0E4
:100B900016C0FA0120813181F7018081918182178D
:100BA00093073CF48D919C911197019711969C931A
:100BB0008E936F5F7F4F22E030E0E20EF31E6017EE
:100BC00071073CF30894A11CB11C12964E5F5F4F55
:100BD000A016B106BCF282DB88E990E06FDB0ADB8D
:100BE000F8DA08DBF6DA85E990E068DB86B396B3DD
:100BF0009470282F227081FF07C09923B9F71092B3
:100C0000C2002093C30004C09093C2001092C3009E
:100C100086B396B39470282F227081FFF9CF992361
:100C2000B9F39093C2002093C300AA24BB246E01A1
:100C30000894C11CD11C8BE090E0A89EF001A99EF5
:100C4000F00DB89EF00D1124E45BFE4F80818823E7
:100C500011F4AA24BB248091BA019091BB01892B85
:100C600021F43CDB84E890E0F7C1A114B10409F061
:100C7000AEC034DB8AE790E021DB80E790E01EDB4A
:100C800086B396B39470282F227081FF07C09923F2
:100C9000B9F71092C2002093C30004C09093C20021
:100CA0001092C30084ED90E30197F1F786B3827050
:100CB0008093C30096B394709093C200882351F53B
:100CC000992341F520E23EE489E190E00197F1F7B4
:100CD00021503040C9F786B382708093C30096B329
:100CE00094709093C2008823A9F4992399F459DA57
:100CF000F5DA80E690E0D8DA86B396B39470282FC0
:100D0000227081FFF9CF9923B9F39093C200209309
:100D1000C300EFCC8091C300882309F458C0DEDA09
:100D200080E590E0CBDA55DA80E090E006C084E21E
:100D300094EF0197F1F781E090E0E9DA892BB9F7B8
:100D400030DA2FDA2EDA8BE090E09093BD018093B9
:100D5000BC018301EE24FF24B401C80199D100979E
:100D600021F4F092BD01E092BC010894E11CF11C59
:100D70003AE0E316F10421F0055F1F4F892B61F77C
:100D8000ADDA87E490E09ADAE091BC01F091BD0120
:100D9000EB30F10521F48DE390E090DA0EC0EE0F18
:100DA000FF1FEB5CFE4F80819181B3E0880F991F9C
:100DB000BA95E1F78F589F4F77DA20E23EE489E158
:100DC00090E00197F1F721503040C9F752CF86B338
:100DD00096B39470282F227081FFF9CF9923B9F32D
:100DE0009093C2002093C30079DAF501EE0FFF1F44
:100DF000EB5CFE4F80819181E3E0880F991FEA95BB
:100E0000E1F78F589F4F50DA5D9BFECF8AE08CB997
:100E1000F501EE0FFF1FEF5DFE4F4AE050E0B60117
:100E20008081918153D1C6013FDA89E390E046DAAF
:100E300062E088E05CDA5D9BFECF8EE38CB986B31E
:100E400096B39470282F227081FF07C09923B9F7B9
:100E50001092C2002093C30004C09093C20010926D
:100E6000C30086EA9EE00197F1F786B396B39470CB
:100E7000282F227081FFF9CF9923B9F39093C200F4
:100E80002093C3002BDA2091BA013091BB012832A4
:100E9000310524F0C90168E270E003C088E290E007
:100EA000B90143D1AB015D9BFECF8EEF8CB95D9B49
:100EB000FECF8CE78CB95D9BFECF81E08CB95D9B4A
:100EC000FECF81E08CB95D9BFECF1CB8F501EE0F23
:100ED000FF1FEF5DFE4F608171816217730729F478
:100EE0005D9BFECF88E28CB90BC0CB01489FB0015F
:100EF000499F700D589F700D11245D9BFECF6CB9FA
:100F000062E081E0F4D9D501AA0FBB1FFD01EF5DBE
:100F1000FE4F208131818091BA019091BB01281749
:100F2000390721F481E390E0C9D915C0A251BF4F20
:100F30004AE050E0B6018D919C91C8D05D9BFECFF8
:100F400083E28CB9C601B0D962E088E0D0D95D9B5C
:100F5000FECF8EE38CB986B396B39470282F22709F
:100F600081FF07C09923B9F71092C2002093C300F4
:100F700004C09093C2001092C30086EA9EE00197DD
:100F8000F1F786B396B39470282F227081FFF9CFC2
:100F90009923B9F39093C2002093C3009FD98BE2A9
:100FA00090E08CD9F501EE0FFF1FE652FF4F4AE0AB
:100FB00050E0B6018081918189D0C60175D95D9BD1
:100FC000FECF8AE08CB986E290E078D9F501EE0F89
:100FD000FF1FE35FFE4F4AE050E0B6018081918140
:100FE00075D0C60161D984ED90E30197F1F762E015
:100FF00088E07DD95D9BFECF8EE38CB986B396B336
:101000009470282F227081FF07C09923B9F710929E
:10101000C2002093C30004C09093C2001092C3008A
:1010200086EA9EE00197F1F786B396B39470282F75
:10103000227081FFF9CF9923B9F39093C2002093D6
:10104000C3000894A11CB11C9AE0A916B1040CF4C9
:10105000F2CDAA24BB24EFCD31D981E090E02B96CC
:101060000FB6F894DEBF0FBECDBFDF91CF911F91B9
:101070000F91FF90EF90DF90CF90BF90AF909F9037
:101080008F907F906F905F904F903F902F9008953A
:10109000FB01DC018D91019080190110D9F3990BAE
:1010A0000895FB01DC0101900D920020E1F7089505
:1010B000FB01DC014150504030F08D9101908019CE
:1010C00019F40020B9F7881B990B0895FB019F01C3
:1010D000E8944230BCF04532ACF44A3029F497FB36
:1010E0001EF4909581959F4F642F772731D0805DB6
:1010F0008A330CF0895D8193CB010097A9F716F430
:101100005DE251931082C90100C0DC01FC01672F30
:1011100071917723E1F7329704C07C916D937083CE
:101120006291AE17BF07C8F3089597FB092E0726F3
:101130000AD077FD04D00CD006D000201AF47095A8
:1011400061957F4F0895F6F7909581959F4F08958B
:10115000AA1BBB1B51E107C0AA1FBB1FA617B707DD
:1011600010F0A61BB70B881F991F5A95A9F78095F9
:0A1170009095BC01CD010895FFCF5A
:10117A0062616473746172740062616473746F7023
:10118A0000776967676C6573006C6566747900003F
:10119A0000626F6F6D65720000666C657879000099
:1011AA000073617563790000006665656C6572009D
:1011BA0000776869746579000068616E6479000077
:1011CA00006E617374790000006372617A790000BD
:0211DA00000013
:00000001FF
